:07000000020358121A23321B
:01000B0032C2
:040013001215F5329B
:01001B0032B2
:0100230032AA
:01007000058A
:100080004D503320506C6179657220312E30346FC1
:10009000004D503320506C617965722020205665E8
:1000A0007273696F6E20312E30346F202028627990
:1000B0002044572026204146292D2D2D2D2D2D2D34
:1000C0002D2D2D2D2D2D2D2D2D2D2D2D2D2D2D2D60
:1000D0002D2D2D2D2D2D2D2D2D2D2D2D2D2D2D2D50
:1000E0002D00202020202020202020202020202023
:1000F0002020202020202020202020202020202000
:1001000020202020202020202020004469736B3AEA
:10011000002A2A2052454144204552524F52204F36
:1001200052204E4F204449534B202A2A00547261DA
:10013000636B733A004469736B3A2A2A204E4F204E
:100140004D50332D4344202A2A0020417274697394
:10015000743A2000205469746C653A2020002043D2
:100160006F6D6D656E743A0020416C62756D3A205A
:10017000200020596561723A202020002046696CD9
:10018000653A2020200052454144204552524F52AA
:10019000008253746F7020000B506C617920000C4A
:1001A0005061757365000D456A656374004F4F704B
:1001B000656E20004C4C6F61642000524E4400205C
:1001C0002020004344524F4D3A002A2A20444556ED
:1001D000494345204944454E5449465920455252C9
:1001E0004F52202A2A002A2A204E4F204F522049BF
:1001F0004E434F4D50415449424C45204344524F89
:100200004D202A2A00032A2A4944454641494C2DBB
:100210003E52455345542A2A0052656164696E670F
:10022000204D50332D5461672773202E2E2E0052FF
:10023000414D3A200052414D3A204F4B2120202081
:100240000052414D3A204552524F522100444543FD
:100250004F4445523A204D4153004445434F444595
:10026000523A204E4F5420464F554E4421212100F2
:10027000044D415320494E4954204552524F52009B
:10028000032A2A204D4153205245494E4954202AE1
:100290002A005254433A20464F554E44005254438C
:1002A0003A204E4F5420464F554E4400465245206A
:1002B0003332203438203536203634203830203957
:1002C00036313132313238313630313932323234FE
:1002D0003235363332303338344552524652452067
:1002E000333220343020343820353620363420382C
:1002F00030203936313132313238313630313932DD
:10030000323234323536333230455252465245203D
:10031000203820313620323420333220343020341B
:1003200038203536203634203830203936313132D5
:100330003132383134343136304552523434343835
:100340003332525332323234313652533131313208
:1003500020385253534A444D75816374FF12152956
:10036000740090007093F525D2AF12175C1211E063
:1003700074FF121529121AA974031218D4121650F8
:10038000121A739000801218E074041218D4740AC0
:10039000121BA8121686740B121BA8121A00740CDA
:1003A000121BA812157674031218D4740D121BA810
:1003B00012142B9011D412174F78007900121217D3
:1003C000121A987520FF7535007536009011B0121D
:1003D000174F7800790012121774FF1214A7120831
:1003E0007E74041218D47402121BA8120DCF120EC0
:1003F00023753100753200120E4FE5314532701E03
:100400007402121BA874041218D49001351218E05B
:10041000900135121AC0D2002000FD0204C57403F9
:100420001218D490012D1218E0740275F01E121BE0
:100430009790012D121AC0A831A9327A007B0012C0
:1004400014DD900000E01218D4121B79A3E01218FA
:10045000D4121B79A3E01218D4121B7975C9007548
:10046000C804E532F4F5CAF5CCE531F4F5CBF5CDA9
:10047000740E121BA8900219121AC075330075343D
:1004800001120C2A0534E53470020533D3E53195A9
:100490003350EEC3E532953450E7753300753401BF
:1004A0001215C2D3E5319533500DC3E53295345062
:1004B00006753300753401020542B22AD2061208CD
:1004C0007E1208872275816312087EC2AFC290D265
:1004D00091D2927420900000F0A3F0A3F075330045
:1004E0007534011215A3121A63121A7374051218C7
:1004F000D4740312101C9011BC12174F78007900AD
:100500001212179011A412174F78007900121217C7
:10051000740412101CD20030000F9011D412174F27
:100520007800790012121740EE740512101C901119
:100530009812174F7800790012121761B33028858E
:10054000C228121540E532C399E53198400BE849BD
:1005500060078934883312087E7520FF754701C310
:10056000E535953340127010C3E536953440097077
:1005700007020592D22880CA1209E71208DE120A81
:10058000EB7548007549038533358534367405129B
:1005900018D4202811740012101C1547E547700666
:1005A00012095F75472020060291BA20010B9002C4
:1005B000801218E0D201121A1930002030032C30BA
:1005C00002663004193005533007A93028C41214CC
:1005D000D1120650E5200470B9020628A13DC3E5FA
:1005E000349409F534E5339400F533C3E5349401CC
:1005F000F534E5339400F533C3E5329534E53195B0
:10060000334008E533700AE53470068531338532AE
:1006100034E52004600312087EA142C3E5343409A6
:10062000F534E5333400F533C3E5343401F534E50E
:10063000333400F533C3E5329534E5319533400862
:10064000E533700AE534700675340175330080C1F6
:1006500012088712158F1215A374051218D41209E7
:100660005F754700740112101C120D06C290D291E2
:10067000D292A3E0FBA3E0FAA3E0F9A3E0F8883A62
:10068000893B8A3C8B3DA3E0FBA3E0FAA3E0F9A3FE
:10069000E0F8120FB2E53DC33BF541E53C3AF540C9
:1006A000E53B39F53FE53A38F53EC2A8A83AA93B03
:1006B000AA3CAB3D7D207E007F00D290D291D292A9
:1006C000120F655039C0E074021218D47445121824
:1006D000D4743A1218D4D0E0121910C0E074211268
:1006E00018D4740875F023121B977445121B797483
:1006F0003A121B79D0E0121BCC74FF121529752316
:1007000000752200C208D2A81207ED1207EDC3E55A
:1007100041953DFDE540953CE53F953BE53E953AED
:10072000501C30A816C3ED3410C333C333C3332079
:100730000802D2E7F524C2093009FD02078C20081F
:10074000077E00D20802074C7E80C208C00612193C
:1007500090740112101CD006EE652254807039C3CB
:10076000E5229547C3940C400712095FE522F5473F
:1007700030001930071630031330021030041330E4
:10078000051330010A2006C491BA80C0C2A8220213
:100790000849020828020807A83AA93BAA3CAB3D31
:1007A0007D107F00D290D291D292120F655039C045
:1007B000E074021218D474451218D4743A1218D482
:1007C000D0E0121910C0E074211218D4740875F02A
:1007D00023121B977445121B79743A121B79D0E0CF
:1007E000121BCC74FF1215291207EDE10EE53DC373
:1007F0003410F53DE53C3400F53CE53B3400F53B79
:10080000E53A3400F53A22C2A8E53DC33450F53D3F
:10081000E53C3400F53CE53B3400F53BE53A34007B
:10082000F53A7520FF0206AAC2A8E53DC39450F52B
:100830003DE53C9400F53CE53B9400F53BE53A94FE
:1008400000F53A7520FF0206AAC2A8754701740593
:100850001218D485FF2074081215291547E5477032
:100860000B12095F740212101C754720E52004600A
:10087000E585FF20D2A8740112101C02074C7420D9
:10088000F54AF54BF54C22C000C001C002C003C0C0
:1008900004C005C006C007302833302A30E5CCF448
:1008A000F9E5CDF4F84960DF7AFF7BFDC2AFC29075
:1008B000D291D2921214DD90FFFDE0F54AA3E0F54B
:1008C0004BA3E0F54CD290D291D292D2AFD007D0C8
:1008D00006D005D004D003D002D001D00022853349
:1008E00037853438C3E5349404F534E5339400F5A2
:1008F0003375390AE539121BA8C3E5349401E53391
:100900009400400EC3E5329534E53195334003122F
:1009100009420539C3E5343401F534E5333400F5D3
:1009200033E539C3940F700C0539740E121B8674AD
:100930000D121B79E539C3941940B98537338538D1
:100940003422120A7E900000C2AFC290D291D2929D
:1009500075F027121B21D290D291D292D2AF22747D
:10096000011218D4758300854982754828C2AFC228
:1009700090D291D292E0D290D291D292D2AF700521
:1009800090000380E81218D4A31548E54870DE05EE
:1009900049758300854982C2AFC290D291D292E05C
:1009A000D290D291D292D2AF7003754903D290D235
:1009B00091D292D2AF227404121BA804121BA87405
:1009C00007121BA804121BA87406121BA890017C16
:1009D000121AC0120D067409120FE8121AEED29004
:1009E000D291D292D2AF22C2AFC290D291D2921201
:1009F0000D06E0F5263035BE7404121BA890014A9E
:100A0000121AC0120D067427120FE875F01E121B81
:100A1000217405121BA8900154121AC0120D0674FD
:100A200009120FE875F01E121B217406121BA89004
:100A3000015E121AC0120D067467120FE875F01EDF
:100A4000121B217407121BA8900168121AC0120D04
:100A5000067445120FE875F01E121B217408121B54
:100A6000A8900172121AC0120D067463120FE87575
:100A7000F004121B21D290D291D292D2AF227A00EE
:100A80007B00C2AFC290D291D292120BA2A934A81D
:100A9000331214DD120BA2120D06E0F52620350EDE
:100AA000120D067409120FE8120B85020ADB120DF3
:100AB000067427120FE87F0F120BD9120BAF120D1D
:100AC000067409120FE87F1D120BD9120BA2120D2A
:100AD000067467120FE87F1C120BD98A838B82740D
:100AE00000F0D290D291D292D2AF227A007B00C293
:100AF000AFC290D291D292A934A8331214DD120D54
:100B000006E0F526203511120B68120D0674091245
:100B10000FE8120B85020B55120D067427120FE811
:100B20007F1D120BD9120BAF120D067409120FE8BC
:100B30007F1D120BD9120BA2120D067467120FE85B
:100B40007F1C120BD9120BAF120D067445120FE861
:100B50007F1D120BD9120BC48A838B827400F0D2D2
:100B600090D291D292D2AF228A838B827446F0A324
:100B70007469F0A3746CF0A37465F0A3743AF0A3E5
:100B8000AA83AB8222A883A98288838982E060112C
:100B9000A3A883A9828A838B82F0A3AA83AB8280D5
:100BA000E8228A838B827420F0A3AA83AB82228AF4
:100BB000838B827420F0A3742DF0A37420F0A3AA79
:100BC00083AB82228A838B827420F0A3740BF0A300
:100BD0007420F0A3AA83AB8222A883A982C3E582F2
:100BE0003FF582E5833400F583E070027420C394FE
:100BF00020700A120C1B1FEF04601F80EC0F88830B
:100C00008982E070027420A3A883A9828A838B82E0
:100C1000F0A3AA83AB821FEF70E4221582C0E0E547
:100C2000820470021583D0E02222120D06C290D2F7
:100C300091D292E0F5262034F07405120FE8E0FB23
:100C4000A3E0FAA3E0F9A3E0F8EBC39480FBEA94F5
:100C500000FAE99400F9E89400F8120FB2120D06B8
:100C6000A3C3E03BFBA3E03AFAA3E039F9A3E028F1
:100C7000F8ECC0E0EDC0E07D027E007F00120F6561
:100C80004073D0E0FDD0E0FCEDC33400F582EC34DD
:100C900000F583D290D291D292E0A3C394547046CF
:100CA000E0A3C39441703FE0A3C394477038AC8382
:100CB000AD82120D067409120FE8AE83AF82787D03
:100CC000D290D291D2928C838D82E0A3AC83AD82FC
:100CD000C290D291D2928E838F82F0A3AE83AF82E4
:100CE00018E870DCD235D234120D06C290D291D2FF
:100CF00092E526F022D0E0D0E09001861218E09034
:100D00000186121AC022C3E53475F089A4F58285E4
:100D1000F083C3E53375F089A4C32583F583228569
:100D20002982852A83A3A3D290D291D292E0FBA3F9
:100D3000E0FAA3E0F9A3E0F8A3A3A3A3A3E0FFA331
:100D4000E0FEA3E0FDA3E0FCB106C290D291D292F6
:100D50007400F0A3EBF0A3EAF0A3E9F0A3E8F0A39A
:100D6000EFF0A3EEF0A3EDF0A3ECF0A3AF82AE831F
:100D7000852982852A83D290D291D2927420120F33
:100D8000E8E0F8A3D290D291D292E0AD82AC838F0A
:100D9000828E83C290D291D292F0C3943B600EA314
:100DA000AF82AE838D828C83A318E870D78F828E3A
:100DB00083C290D291D2927400F022900111121845
:100DC000E0900111121AC0D2002000FD0204C5906B
:100DD000010B1218E090010B121AC07542FF30008F
:100DE000EB74FF1215299011D412174F1212171518
:100DF00042E54260C640E7780079007A007B107DCA
:100E0000017E087F00120F6540B1D290D291D2923C
:100E10009008487400F09008281218ED90082812E5
:100E20001AEE22900884E0FBA3E0FAA3E0F9A3E025
:100E3000F8120FB2EB04FD90088CE0FBA3E0FAA3DC
:100E4000E0F9A3E0F87E107F00120F65403C22908D
:100E50001000D290D291D292E0FD602DA3A3E0FBCE
:100E6000A3E0FAA3E0F9A3E0F8A3A3A3EDFEA31E79
:100E7000EE70FBED135001A3858227858328120EA7
:100E80008C85278285288380C922A1BB90F00088A9
:100E90002B892C8A2D8B2E7D017EF07F00120F6511
:100EA00040E890F000740A120FE8D290D291D292EA
:100EB000E0FBA3E0FAA3E0F9A3E0F8120FB28B3055
:100EC000120EDDA82BA92CAA2DAB2E120FF1882B08
:100ED000892C8A2D8B2E1530E53070E42290F0009D
:100EE000A82BA92CAA2DAB2E7D017EF07F00120F1E
:100EF00065409790F00085822985832AD290D2910F
:100F0000D292E0605FF52FE583C394F850567419D0
:100F1000120FE8E07041852982852A837420120F20
:100F2000E8E0F9A3E0C3942E6008A319E970F50284
:100F30000F57A3E0C3944D701EA3E0C394507017E5
:100F4000A3E0C3943370100532E532700205318599
:100F50003234853133B11F852982852A83E52F12EA
:100F60000FE8809222C000C001C002C003C004C0CC
:100F700005C006C007120F8BD007D006D005D004DD
:100F8000D003D002D001D000400122754DA8754E8B
:100F900000884F89508A518B5275530075540075E3
:100FA00055008D56755700755800EFF8EEF912127E
:100FB000172212100812100812100812100812102E
:100FC0000812100812100812100812100812100847
:100FD000121008C3121015C3121015C3121015C336
:100FE000121015C3121015222582F58250020583B6
:100FF0002274012BFB501074012AFA500A74012943
:10100000F95004740128F822C3E813F8E913F9EA47
:1010100013FAEB13FBEC13FCED13FD229001917519
:10102000F007C3A4C33582F582E5F03583F58374F8
:10103000021218D4C082C0837400931218D4C2AFB5
:10104000C290D291D292900000E01218D4A3E01284
:1010500018D4A3E01218D4740875F015121B972049
:101060002A0B74201218D49001BF0210757452120A
:1010700018D49001BB121AC0D290D291D292D2AFA2
:10108000740875F023121B97D083D082A3121AC064
:10109000E54A1218D4E54B1218D4E54C1218D47452
:1010A0000875F01F121B97E54A121B79E54B121BBE
:1010B00079E54C121B79C0E0202803D0E0223029CA
:1010C0003B740875F019121B9774201218D474A081
:1010D00075F0031217F574A0121828121910121BBC
:1010E000CC743A1218D4121B7974A075F00212173E
:1010F000F574A0121828121910121BCC74201218A3
:10110000D41218D4740875F00E121B97E55F64FFB3
:10111000546090030C700CE55F54109002DC600387
:101120009002ACE56154F0C31313131375F003A4DC
:10113000C0E0931218D4121B79D0E004C0E09312DF
:1011400018D4121B79D0E004931218D4121B79E53D
:101150006254C0C313131313131390035493121840
:10116000D4121B79E55F546090034C600A900344ED
:101170005420600390033CE561540CC3131375F0D5
:1011800002A4C0E0931218D4121B79D0E004931289
:1011900018D4121B79D0E0221B00000003000000CD
:1011A000000000001B000000020000000000000022
:1011B0001E00000001000000000000001E000000F2
:1011C00000000000000000001200000024000000E9
:1011D000000000000000000000000000000000000F
:1011E000D2B0D293D294D2B1C2B07405121529D222
:1011F000B0742012152922C0E01543E54370121582
:1012000044E544700C1545E5457006854681021499
:1012100017D0E030B1E122754300754400754530C8
:10122000858146C2AFD290D291D292D294D2937598
:1012300080FF75A0FF31F7C29331F7E580D293D2DA
:1012400090D291D292D2AF0020E7D820E3D5C2AF9E
:10125000C290D291D2927580FF75A0FF7580A031A7
:10126000F7C29431F7D294D290C291C292758000A5
:1012700031F7C29431F7D294D290C291D292758054
:101280008031F7C29431F7D294C290C291D2927554
:10129000800031F7C29431F7D294D290D291D29299
:1012A0007580A031F7C29431F7D2947D06C00078E2
:1012B0004D0212B9D000021351C2AFD290D291D2D6
:1012C000927580FF75A0FF31F7C29331F7E580D2A8
:1012D00093D290D291D292D2AF0020E7DC20E0D41A
:1012E00030E3D6C2AFC290C291C292E6FE08E6FFDA
:1012F000088E808FA031F7C29431F7D294DDECD004
:1013000000D290D291D2927580FF75A0FF31F7C2C2
:101310009331F7E580D29320E3EDD290D291D2922F
:10132000D2AF00C2AFD290D291D2927580FF75A099
:10133000FF31F7C29331F7E580D293D290D291D2A8
:1013400092D2AF0020E7DC20E00720E3267400C340
:1013500022C2AFD290C291C2927580FF75A0FF31B8
:10136000F7C29331F7E580D293D290D291D292D244
:10137000AFD32288828983C2AFD290C291D29275B4
:1013800080FF75A0FF31F7C29331F7AB80D293C2D3
:1013900090C291D2927580FF75A0FF31F7C2933150
:1013A000F7AA80D293C3EB13FBEA13FA50050AEABB
:1013B00070010BEA4B6030C2AFC290C291C292750D
:1013C00080FF75A0FF31F7C29331F7A880A9A0D2A2
:1013D00093D290D291D292D2AF00E8F0A3E9F0A3D9
:1013E000DAD1EB6002DBCCC2AFD290D291D292754F
:1013F00080FF75A0FF31F7C29331F7E580D293D219
:1014000090D291D292D2AF0020E7DC20E01B20E303
:10141000047400C32261779002051218E031E07471
:10142000FF12152974011218D461519001C31218CA
:10143000E09001C3121AC09011D412174F780079AE
:1014400000511790119812174F780079005117909A
:1014500011D412174F7800790051179011C8121744
:101460004F7800790051174024D290D291D29290B7
:101470000000E0541FC3940570209000247400F015
:101480009000081218ED900008121AEE229001CA7E
:101490001218E09001CA121AC0229001E61218E058
:1014A0009001E61218E022754DBB754E00F54F75A0
:1014B00050007551FF7552FF7553007554007555F6
:1014C000007556007557007558007800790051175F
:1014D000227410C0E091A7D0E01470F722C082C03F
:1014E00083C0E08A838B827E277F107E037FE87E25
:1014F000007F6412150F7E007F0A12150F7E007F99
:101500000112150FAA83AB82D0E0D083D08222755E
:10151000F030C3E99FE89E400BC3E99FF9E89EF8CD
:1015200005F080EEE5F0F0A32212153115E070F918
:1015300022C0E074FF14000000000070F8D0E02228
:1015400078007900E54A540F75F064121564E54B94
:10155000540F75F00A121564E54C540F75F0011222
:101560001564222260FDC0E0C3E935F0F9E83400DB
:10157000F8D0E01480EE74A0121828B39229302914
:1015800007900292121AC02290029D121AC02230B5
:10159000290B90159E74A075F00512186B2201009E
:1015A00000000030291B74A07810A93412184A7466
:1015B000A07811A93312184A74A07812A92512181C
:1015C0004A223029FC74A075F0101217F574A0128D
:1015D0001828F53474A075F0111217F574A01218BC
:1015E00028F53374A075F0121217F574A01218289C
:1015F000F525D22922C0D0C0E0C0F07440121828CE
:10160000400BC0E0C3940C4014D0E0522074701220
:10161000182840025220D0F0D0E0D0D022D0E0B440
:101620000A0FE54BF54CE54AF54B7420F54A0216D6
:1016300049B40B05C206021649C0E0E54BF54AE580
:101640004CF54BD0E02430F54CD0F0D0E0D0D02297
:10165000D2AA744075F0FF1217F57520FF227AFFA9
:101660007BFF8A838B82E0C3987008E9F0DBF3DAB2
:10167000EFC322D32278FF79FF88838982F0D9F9DA
:10168000D8F52202173790022F1218E090022F127D
:101690001AC0C290D291D2927400D175D290D291D8
:1016A000D292D175780079F0D15E40D7743112189A
:1016B000D4121B7978F0790FD15E40C774321218BA
:1016C000D4121B79780F79FFD15E406B74331218F6
:1016D000D4121B7978FF79FFD15E405BC290D29122
:1016E000D292780079F0D15E404D74311218D41244
:1016F0001B7978F0790FD15E403D74321218D41204
:101700001B79780F79FFD15E402D74331218D412F3
:101710001B7978FF79FFD15E401D74021218D474D2
:101720000A121B869002351218E0900235121AC078
:10173000D290D291D2922274021218D4740A121B3F
:10174000869002411218E0900241121AC080FE7F7A
:101750000C784D740093A3F608DFF822D2B5D2B40A
:1017600030B4FD22000000000000000022D2B5D2FB
:10177000B430B51030B4FD30B50AF164C2B5F164CF
:10178000C2B4C322D322C2B5F164D2B4F16430B47E
:10179000FDD2B522C0F075F0083392B5F164D2B431
:1017A00030B4FDF164C2B4F164D5F0EDD2B5F164AA
:1017B000D2B4F16430B4FDA2B5C2B4D0F022D2B537
:1017C000C0F075F008F164D2B4F16430B4FDA2B594
:1017D00033C2B4D5F0EFD0F022C2B5F164D2B4F187
:1017E0006430B4FDC2B422D2B5F164D2B4F1643035
:1017F000B4FDC2B422C2AAF16D4048C2E0F19440E7
:1018000042E5F0121794403B121786C3D2AA22C2B7
:10181000AA12176D402DC2E01217944026E5F0126F
:101820001794401FC3D2AA22C2AA12176D4014D225
:10183000E0121794400D1217BE1217E7121786C355
:10184000D2AA22121786D3D2AA22C2AA12176D4098
:10185000F2C2E012179440EBE812179440E5E91247
:10186000179440DF121786C3D2AA22C2AA12176D9C
:1018700040D1C2E012179440CA74009312179440EA
:10188000C2A3D5F0F4121786C3D2AA22C2AA121795
:101890006D40B0C2E012179440A97400E012179492
:1018A00040A1A3D5F0F4121786C3D2AA22C2AA126D
:1018B000176D408FD2E012179440881217BEC0E017
:1018C0001217D91217BEF5F01217E7121786D0E0DB
:1018D000C3D2AA22C0E0F5F074201217F5D0E0229E
:1018E0007400934400600511D4A380F4227400E0D6
:1018F000440060F811D4A380F422540F2430C0E0D7
:10190000C3943A4006D0E02407C0E0D0E011D422CE
:10191000C0E0C411FAD0E0C0E011FAD0E022689E25
:10192000620000680FCD68A0000002036DD9E800D6
:1019300005ECF5000C68047568304168308168F08A
:101940000000010FF668F00000010FF790193E74D7
:101950003A75F007116B743A75F069110F743A110A
:10196000ADC0F0121BCCD0E0121BCC7420121B793E
:10197000901945743A75F007116B743A75F0691156
:101980000F743A11ADC0F0121BCCD0E0121BCC2268
:10199000901938743A75F003116B743A75F0691147
:1019A0000F743A11ADF55F85F06090193B743A758C
:1019B000F003116B743A75F069110F743A11ADF5BB
:1019C0006185F06222D297D29575D55D90191E740B
:1019D0003A75F005116B4026901923743A75F0039F
:1019E000116B401A901926743A75F00F116B400E66
:1019F000901935743A75F003116B4002C322D3225B
:101A000031C5400990024D121AC0314C2290025A41
:101A1000121AC090027011E0227409121B8631C59F
:101A200040EB22C083C082C0E0C0D08522838523E2
:101A300082E0A3F586E524C395837002D209E5AA66
:101A400030E7FB30B2EB858223858322D0D0D0E013
:101A5000D082D08322001004000004000C0C000887
:101A6000080000901A5F742275F004116BE51012E3
:101A7000152922740075F000121B97900091121A1C
:101A8000C07403121B869000B9121AC07409121B8D
:101A9000869000B9121AC022741975F007121B97AC
:101AA000740875F00B121B4E22901A55742275F0B3
:101AB00005116B901A5A742275F005116B5163224F
:101AC000C2AA12176D40537422C2E0121794404A02
:101AD000740B1217944043740093600B121BDA12BC
:101AE00017944036A380F0121786C3D2AA22C2AA46
:101AF00012176D40257422C2E0121794401C740B1B
:101B00001217944015E0600B121BDA121794400A6A
:101B1000A380F2121786C3D2AA22121786D3D2AAA2
:101B200022C2AA12176D40F27422C2E0121794402A
:101B3000E9740B12179440E2E060D8121BDA121716
:101B40009440D7A3D5F0F1121786C3D2AA22C2AA15
:101B500012176D40C5C0E07422C2E0121794D0E0A5
:101B600040B8C0E0E5F0121794D0E040AD121794F1
:101B700040A8121786C3D2AA22C0E0121BDA75F061
:101B80000B714ED0E022C0E075F009714E74007503
:101B9000F00A714ED0E022C0E0E5F075F00A714E17
:101BA000D0E075F009714E227186C0E09000E251DC
:101BB000C0D0E0718622540F2430C0E0C3943A4074
:101BC00006D0E02407C0E0D0E0717922C0E0C47103
:101BD000B6D0E0C0E071B6D0E022C082C083901BD6
:101BE000E793D083D0822220010203040506070870
:101BF000090A0B0C0D0E0F101112131415161718DD
:101C0000191A1B1C1D1E1F202122232425262728CC
:101C1000292A2B2C2D2E2F303132333435363738BC
:101C2000393A3B3C3D3E3F8041424344454647486C
:101C3000494A4B4C4D4E4F5051525354555657589C
:101C4000595A282F298E5F27616263646566676829
:101C5000696A6B6C6D6E6F7071727374757677787C
:101C6000797A288829C77F7F7F7F7F7F7F7F7F7FEB
:101C70007F7F7F7F7F7F7F7F27277F7F7F7F7F7F24
:101C80007F7F7F7F7F7F7F20E0CCC3945988402275
:101C900063E58BC72D7281CBC73233277588C72C7C
:101CA00031E68D828C89E1F1F0D2D55B9DF9D7F2D6
:101CB00090DCDBCAF3DEF4FBE7F6F5D8D65C78FD02
:101CC000C1F7D95D59FE7ED0EBD2C57B99F8DAD148
:101CD000C0DCDBCAEDDED4FAE8C8EED8C67C8AFCEC
:071CE000DDEFD97D79FE79EB
:00000001FF
